:100000006F28A0008417800484138E010C1C8E00BE
:10001000102003196A28102003196A2810206A2862
:1000200020088E0601308C008D01000820050E0688
:10003000031D08008C0A03198D0F152808008F0175
:100040008E00FF308E07031C8F07031C6A280330C5
:100050008D00DF302D2021288D01E83E8C008D0998
:10006000FC30031C36288C07031833288C076400E7
:100070008D0F33280C183C288C1C40280000402889
:1000800008008E000330442894000F080D02031D61
:100090004B280E080C0204300318013003190230FB
:1000A0001405031DFF306A28103094008D018C0167
:1000B000930C920C031C62280E088C070F0803187F
:1000C0000F0F8D078D0C8C0C910C900C940B5828F5
:1000D00010086A2883130313831264000800831630
:1000E000083085008601831285018601DD290130F3
:1000F0008C0005308400083001200C08A6000D0893
:10010000A70026088C0027088D008F015030412061
:10011000031D8C28A901080026088C0027088D00E3
:100120008F0175304120031D98280130A900080077
:1001300026088C0027088D008F018E304120031D7A
:10014000A4280230A900080026088C0027088D008A
:100150008F01A2304120031DB0280330A900080000
:1001600026088C0027088D008F01BB304120031D1D
:10017000BC280430A90008000530A90008000511BA
:100180008316051183124730860032301F20051177
:100190008316051183123830860032301F20051176
:1001A0008316051183126730860032301F20051137
:1001B0008316051183121830860032301F20051572
:1001C0008316051183124030860032301F2005113E
:1001D0008316051183123830860032301F20051532
:1001E0008316051183122030860032301F2005113E
:1001F0008316051183128730860032301F200515C3
:10020000831605118312860132301F2005118316D3
:1002100005118312A730860032301F200511831686
:10022000051183122030860032301F2005118316FD
:10023000051183128030860032301F20051183168D
:10024000051183124730860032301F2005118316B6
:10025000051183123830860032301F2005118316B5
:10026000051183126730860032301F200511831676
:10027000051183121830860032301F2005158316B1
:10028000051183124030860032301F20051183167D
:10029000051183123830860032301F200515831671
:1002A000051183122030860032301F20051183167D
:1002B000051183128730860032301F200515831602
:1002C00005118312860132301F2005118316051196
:1002D0008312A730860032301F20051183160511C6
:1002E00083122030860032301F200511831605113D
:1002F00083128030860032301F20051183160511CD
:1003000083124730860032301F20051183160511F5
:1003100083123830860032301F20051183160511F4
:1003200083126730860032301F20051183160511B5
:1003300083121830860032301F20051583160511F0
:1003400083124030860032301F20051183160511BC
:1003500083123830860032301F20051583160511B0
:1003600083122030860032301F20051183160511BC
:1003700083128730860032301F2005158316051141
:100380008312860132301F20051183160511831256
:10039000A730860032301F20051183160511831205
:1003A0002030860032301F2005118316051183127C
:1003B0008030860032301F20092A8501860105150C
:1003C00083160511831203308F00E83020200511B9
:1003D0008316051183120130A400A5010130A80085
:1003E0006400093028020318082A2408860024081B
:1003F00092002508930002308E008F015420A40043
:100400001108A50003308F00E8302020A80FF02944
:100410008601BF2829088D00053C031C272A8D0D65
:1004200017228C000D1017228A000C08820002305F
:100430008A000D0882070034BF340034BF34003412
:10044000BF34023428340034BF340034BF34092AA6
:0C0450008501E0308600092A63002C2A98
:02400E00FD3F74
:00000001FF
